Archive member included because of file (symbol)

/opt/ic-dev-env/gcc-arm-none-eabi-4_8-2014q3/bin/../lib/gcc/arm-none-eabi/4.8.4/../../../../arm-none-eabi/lib/armv7-m/libc.a(lib_a-exit.o)
                              /opt/ic-dev-env/gcc-arm-none-eabi-4_8-2014q3/bin/../lib/gcc/arm-none-eabi/4.8.4/../../../../arm-none-eabi/lib/armv7-m/crt0.o (exit)
/opt/ic-dev-env/gcc-arm-none-eabi-4_8-2014q3/bin/../lib/gcc/arm-none-eabi/4.8.4/../../../../arm-none-eabi/lib/armv7-m/libc.a(lib_a-impure.o)
                              /opt/ic-dev-env/gcc-arm-none-eabi-4_8-2014q3/bin/../lib/gcc/arm-none-eabi/4.8.4/../../../../arm-none-eabi/lib/armv7-m/libc.a(lib_a-exit.o) (_global_impure_ptr)
/opt/ic-dev-env/gcc-arm-none-eabi-4_8-2014q3/bin/../lib/gcc/arm-none-eabi/4.8.4/../../../../arm-none-eabi/lib/armv7-m/libc.a(lib_a-init.o)
                              /opt/ic-dev-env/gcc-arm-none-eabi-4_8-2014q3/bin/../lib/gcc/arm-none-eabi/4.8.4/../../../../arm-none-eabi/lib/armv7-m/crt0.o (__libc_init_array)
/opt/ic-dev-env/gcc-arm-none-eabi-4_8-2014q3/bin/../lib/gcc/arm-none-eabi/4.8.4/../../../../arm-none-eabi/lib/armv7-m/libc.a(lib_a-memcpy.o)
                              ./main.o (memcpy)
/opt/ic-dev-env/gcc-arm-none-eabi-4_8-2014q3/bin/../lib/gcc/arm-none-eabi/4.8.4/../../../../arm-none-eabi/lib/armv7-m/libc.a(lib_a-memset.o)
                              /opt/ic-dev-env/gcc-arm-none-eabi-4_8-2014q3/bin/../lib/gcc/arm-none-eabi/4.8.4/../../../../arm-none-eabi/lib/armv7-m/crt0.o (memset)
/opt/ic-dev-env/gcc-arm-none-eabi-4_8-2014q3/bin/../lib/gcc/arm-none-eabi/4.8.4/../../../../arm-none-eabi/lib/armv7-m/libc.a(lib_a-__call_atexit.o)
                              /opt/ic-dev-env/gcc-arm-none-eabi-4_8-2014q3/bin/../lib/gcc/arm-none-eabi/4.8.4/../../../../arm-none-eabi/lib/armv7-m/libc.a(lib_a-exit.o) (__call_exitprocs)
/opt/ic-dev-env/gcc-arm-none-eabi-4_8-2014q3/bin/../lib/gcc/arm-none-eabi/4.8.4/../../../../arm-none-eabi/lib/armv7-m/libc.a(lib_a-atexit.o)
                              /opt/ic-dev-env/gcc-arm-none-eabi-4_8-2014q3/bin/../lib/gcc/arm-none-eabi/4.8.4/../../../../arm-none-eabi/lib/armv7-m/libc.a(lib_a-__call_atexit.o) (atexit)
/opt/ic-dev-env/gcc-arm-none-eabi-4_8-2014q3/bin/../lib/gcc/arm-none-eabi/4.8.4/../../../../arm-none-eabi/lib/armv7-m/libc.a(lib_a-fini.o)
                              /opt/ic-dev-env/gcc-arm-none-eabi-4_8-2014q3/bin/../lib/gcc/arm-none-eabi/4.8.4/../../../../arm-none-eabi/lib/armv7-m/libc.a(lib_a-__call_atexit.o) (__libc_fini_array)
/opt/ic-dev-env/gcc-arm-none-eabi-4_8-2014q3/bin/../lib/gcc/arm-none-eabi/4.8.4/../../../../arm-none-eabi/lib/armv7-m/libc.a(lib_a-__atexit.o)
                              /opt/ic-dev-env/gcc-arm-none-eabi-4_8-2014q3/bin/../lib/gcc/arm-none-eabi/4.8.4/../../../../arm-none-eabi/lib/armv7-m/libc.a(lib_a-atexit.o) (__register_exitproc)
/opt/ic-dev-env/gcc-arm-none-eabi-4_8-2014q3/bin/../lib/gcc/arm-none-eabi/4.8.4/../../../../arm-none-eabi/lib/armv7-m/librdimon.a(rdimon-_exit.o)
                              /opt/ic-dev-env/gcc-arm-none-eabi-4_8-2014q3/bin/../lib/gcc/arm-none-eabi/4.8.4/../../../../arm-none-eabi/lib/armv7-m/libc.a(lib_a-exit.o) (_exit)
/opt/ic-dev-env/gcc-arm-none-eabi-4_8-2014q3/bin/../lib/gcc/arm-none-eabi/4.8.4/../../../../arm-none-eabi/lib/armv7-m/librdimon.a(rdimon-_kill.o)
                              /opt/ic-dev-env/gcc-arm-none-eabi-4_8-2014q3/bin/../lib/gcc/arm-none-eabi/4.8.4/../../../../arm-none-eabi/lib/armv7-m/librdimon.a(rdimon-_exit.o) (_kill)

Memory Configuration

Name             Origin             Length             Attributes
CSM_ECSL_Z1      0x00200000         0x00000024
CSM_RSVD_Z1      0x00200024         0x0000000c
RESETISR         0x00200030         0x00000010         xr
INTVECS          0x00201000         0x000001bc         xr
FLASHLOAD        0x00201200         0x00002e00         xr
FLASH            0x00204000         0x0007bf00         xr
CSM_RSVD_Z2      0x0027ff00         0x000000dc
CSM_ECSL_Z2      0x0027ffdc         0x00000024
C0               0x20000000         0x00004000         xrw
C1               0x20002000         0x00002000         xrw
BOOT_RSVD        0x20004000         0x00000900         xr
C2               0x20004900         0x00001700         xrw
C3               0x20006000         0x00002000         xrw
S0               0x20008000         0x00002000         xrw
S1               0x2000a000         0x00002000         xrw
S2               0x2000c000         0x00002000         xrw
S3               0x2000e000         0x00002000         xrw
S4               0x20010000         0x00002000         xrw
S5               0x20012000         0x00002000         xrw
S6               0x20014000         0x00002000         xrw
S7               0x20016000         0x00002000         xrw
CTOMRAM          0x2007f000         0x00000800         xr
MTOCRAM          0x2007f800         0x00000800         xrw
*default*        0x00000000         0xffffffff

Linker script and memory map

LOAD /opt/ic-dev-env/gcc-arm-none-eabi-4_8-2014q3/bin/../lib/gcc/arm-none-eabi/4.8.4/armv7-m/crti.o
LOAD /opt/ic-dev-env/gcc-arm-none-eabi-4_8-2014q3/bin/../lib/gcc/arm-none-eabi/4.8.4/armv7-m/crtbegin.o
LOAD /opt/ic-dev-env/gcc-arm-none-eabi-4_8-2014q3/bin/../lib/gcc/arm-none-eabi/4.8.4/../../../../arm-none-eabi/lib/armv7-m/crt0.o
LOAD ./bsp.o
LOAD ./cpu.o
LOAD ./flash.o
LOAD ./gpio.o
LOAD ./interrupt.o
LOAD ./ipc.o
LOAD ./ipc_lite.o
LOAD ./ipc_util.o
LOAD ./main.o
LOAD ./ram.o
LOAD ./startup_ccs.o
LOAD ./sysctl.o
LOAD ./system_F28M35H2C.o
LOAD ./systick.o
LOAD ./watchdog.o
START GROUP
LOAD /opt/ic-dev-env/gcc-arm-none-eabi-4_8-2014q3/bin/../lib/gcc/arm-none-eabi/4.8.4/armv7-m/libgcc.a
LOAD /opt/ic-dev-env/gcc-arm-none-eabi-4_8-2014q3/bin/../lib/gcc/arm-none-eabi/4.8.4/../../../../arm-none-eabi/lib/armv7-m/libc.a
LOAD /opt/ic-dev-env/gcc-arm-none-eabi-4_8-2014q3/bin/../lib/gcc/arm-none-eabi/4.8.4/../../../../arm-none-eabi/lib/armv7-m/libm.a
LOAD /opt/ic-dev-env/gcc-arm-none-eabi-4_8-2014q3/bin/../lib/gcc/arm-none-eabi/4.8.4/../../../../arm-none-eabi/lib/armv7-m/librdimon.a
END GROUP
                0x00000400                STACK_SIZE = 0x400
                0x00000100                HEAP_SIZE = 0x100

.resetisr       0x00200030       0x10
 *(.resetisr)
 .resetisr      0x00200030       0x10 ./startup_ccs.o
                0x00200030                __reset__
                0x00200040                . = ALIGN (0x4)

.isr_vector     0x00201000      0x1b0
 *(.isr_vector)
 .isr_vector    0x00201000      0x1b0 ./startup_ccs.o
                0x00201000                g_pfnVectors
                0x002011b0                . = ALIGN (0x4)
                0x00201000                __vectors_start = LOADADDR (.isr_vector)

.eh_frame       0x002011b0        0x4
 .eh_frame      0x002011b0        0x0 /opt/ic-dev-env/gcc-arm-none-eabi-4_8-2014q3/bin/../lib/gcc/arm-none-eabi/4.8.4/armv7-m/crtbegin.o
 .eh_frame      0x002011b0        0x4 /opt/ic-dev-env/gcc-arm-none-eabi-4_8-2014q3/bin/../lib/gcc/arm-none-eabi/4.8.4/armv7-m/crtend.o

.ARM.extab      0x002011b4        0x0
 .ARM.extab     0x002011b4        0x0 /opt/ic-dev-env/gcc-arm-none-eabi-4_8-2014q3/bin/../lib/gcc/arm-none-eabi/4.8.4/../../../../arm-none-eabi/lib/armv7-m/crt0.o

.ARM.exidx      0x002011b4        0x8
 .ARM.exidx     0x002011b4        0x8 /opt/ic-dev-env/gcc-arm-none-eabi-4_8-2014q3/bin/../lib/gcc/arm-none-eabi/4.8.4/../../../../arm-none-eabi/lib/armv7-m/crt0.o

.text           0x00204000     0x43a0
                0x00204000                . = ALIGN (0x4)
 *(.text)
 .text          0x00204000        0x0 /opt/ic-dev-env/gcc-arm-none-eabi-4_8-2014q3/bin/../lib/gcc/arm-none-eabi/4.8.4/armv7-m/crti.o
 .text          0x00204000       0x54 /opt/ic-dev-env/gcc-arm-none-eabi-4_8-2014q3/bin/../lib/gcc/arm-none-eabi/4.8.4/armv7-m/crtbegin.o
 .text          0x00204054       0x74 /opt/ic-dev-env/gcc-arm-none-eabi-4_8-2014q3/bin/../lib/gcc/arm-none-eabi/4.8.4/../../../../arm-none-eabi/lib/armv7-m/crt0.o
                0x00204054                _mainCRTStartup
                0x00204054                _start
 .text          0x002040c8      0x10c ./bsp.o
                0x002040f0                assert_failed
                0x002040f4                Delay
                0x00204120                configure_gpio
                0x0020413c                enableLED
                0x00204150                disableLED
                0x00204164                configure_sysclock
                0x00204180                configure_systick
                0x002041b8                SysTick_Handler
 .text          0x002041d4       0x80 ./cpu.o
                0x002041d4                CPUcpsid
                0x002041e8                CPUprimask
                0x00204200                CPUcpsie
                0x00204214                CPUwfi
                0x00204224                CPUbasepriSet
                0x0020423c                CPUbasepriGet
 .text          0x00204254       0x40 ./flash.o
                0x00204254                FlashGainPump
                0x00204278                FlashLeavePump
 .text          0x00204294      0x990 ./gpio.o
                0x002043cc                GPIODirModeSet
                0x00204444                GPIODirModeGet
                0x002044a0                GPIOIntTypeSet
                0x00204548                GPIOIntTypeGet
                0x002045c0                GPIOPadConfigSet
                0x00204694                GPIOPadConfigGet
                0x00204710                GPIOPinIntEnable
                0x0020473c                GPIOPinIntDisable
                0x00204768                GPIOPinIntStatus
                0x00204798                GPIOPinIntClear
                0x002047b8                GPIOPortIntRegister
                0x002047e0                GPIOPortIntUnregister
                0x00204804                GPIOPinRead
                0x00204828                GPIOPinWrite
                0x00204850                GPIOPinTypeCAN
                0x0020487c                GPIOPinTypeGPIOInput
                0x002048a8                GPIOPinTypeGPIOOutput
                0x002048d4                GPIOPinTypeGPIOOutputOD
                0x00204900                GPIOPinTypeI2C
                0x0020492c                GPIOPinTypeSSI
                0x00204958                GPIOPinTypeTimer
                0x00204984                GPIOPinTypeUART
                0x002049b0                GPIOPinTypeUSBDigital
                0x002049dc                GPIOPinTypeUSBAnalog
                0x00204a08                GPIOPinTypeEPI
                0x00204a34                GPIOPinConfigure
                0x00204b04                GPIOPinConfigureCoreSelect
                0x00204b58                GPIOPinLockStatus
                0x00204b80                GPIOPinLock
                0x00204bd4                GPIOPinUnlock
 .text          0x00204c24      0x4ec ./interrupt.o
                0x00204c2c                IntMasterEnable
                0x00204c3c                IntMasterDisable
                0x00204c4c                IntFlashVTable
                0x00204c70                IntRAMVTable
                0x00204c94                IntRegister
                0x00204cf0                IntUnregister
                0x00204d14                IntPriorityGroupingSet
                0x00204d44                IntPriorityGroupingGet
                0x00204d8c                IntPrioritySet
                0x00204dec                IntPriorityGet
                0x00204e20                IntEnable
                0x00204ee4                IntDisable
                0x00204fa8                IntPendSet
                0x00205054                IntPendClear
                0x002050ec                IntPriorityMaskSet
                0x00205100                IntPriorityMaskGet
 .text          0x00205110      0xa20 ./ipc.o
                0x00205110                IPCMInitialize
                0x002051b8                IpcPut
                0x00205240                IpcGet
                0x002052b0                IPCMtoCDataRead
                0x00205308                IPCMtoCDataRead_Protected
                0x00205364                IPCMtoCSetBits
                0x002053a4                IPCMtoCSetBits_Protected
                0x002053e4                IPCMtoCClearBits
                0x00205424                IPCMtoCClearBits_Protected
                0x00205464                IPCMtoCDataWrite
                0x002054a8                IPCMtoCDataWrite_Protected
                0x002054ec                IPCMtoCBlockRead
                0x00205550                IPCMtoCBlockWrite
                0x0020559c                IPCMtoCBlockWrite_Protected
                0x002055e8                IPCMtoCFunctionCall
                0x00205620                IPCMtoCSendMessage
                0x0020565c                IPCCtoMDataWrite
                0x002056b4                IPCCtoMDataWrite_Protected
                0x00205724                IPCCtoMDataRead
                0x00205780                IPCCtoMDataRead_Protected
                0x002057dc                IPCCtoMSetBits
                0x0020582c                IPCCtoMSetBits_Protected
                0x00205894                IPCCtoMClearBits
                0x002058f0                IPCCtoMClearBits_Protected
                0x00205964                IPCCtoMBlockRead
                0x002059c8                IPCCtoMBlockWrite
                0x00205a60                IPCCtoMBlockWrite_Protected
                0x00205b10                IPCCtoMFunctionCall
 .text          0x00205b30      0xa20 ./ipc_lite.o
                0x00205b30                IPCLiteMtoCGetResult
                0x00205b84                IPCLiteMtoCDataRead
                0x00205bf8                IPCLiteMtoCSetBits
                0x00205c80                IPCLiteMtoCSetBits_Protected
                0x00205d08                IPCLiteMtoCClearBits
                0x00205d90                IPCLiteMtoCClearBits_Protected
                0x00205e18                IPCLiteMtoCDataWrite
                0x00205e8c                IPCLiteMtoCDataWrite_Protected
                0x00205f00                IPCLiteMtoCFunctionCall
                0x00205f68                IPCLiteMtoCBootBranch
                0x00205fc0                IPCLiteCtoMDataRead
                0x00206054                IPCLiteCtoMSetBits
                0x0020610c                IPCLiteCtoMSetBits_Protected
                0x002061dc                IPCLiteCtoMClearBits
                0x0020629c                IPCLiteCtoMClearBits_Protected
                0x00206374                IPCLiteCtoMDataWrite
                0x0020641c                IPCLiteCtoMDataWrite_Protected
                0x002064dc                IPCLiteCtoMFunctionCall
 .text          0x00206550      0x270 ./ipc_util.o
                0x00206550                IPCCtoMFlagAcknowledge
                0x00206574                IPCCtoMFlagBusy
                0x002065a0                IPCMtoCFlagBusy
                0x002065cc                IPCMtoCFlagSet
                0x002065f0                IPCMtoCFlagClear
                0x00206614                IPCMtoCSharedRamConvert
                0x0020664c                IPCMtoCBootControlSystem
 .text          0x002067c0       0x48 ./main.o
                0x002067c0                main
 .text          0x00206808      0x194 ./ram.o
                0x00206808                RAMMReqSharedMemAccess
                0x0020686c                RAMControlInitM1MsgRam
                0x00206904                RAMControlInitL0L3Ram
 .text          0x0020699c      0x124 ./startup_ccs.o
                0x0020699c                Reset_Handler
                0x00206a30                NMI_Handler
                0x00206a40                MemManage_Handler
                0x00206a54                HardFault_Handler
                0x00206a68                BusFault_Handler
                0x00206a7c                UsageFault_Handler
                0x00206a94                FLASHCtrl_IRQHandler
                0x00206a94                DebugMon_Handler
                0x00206a94                CTOMIPC2_IRQHandler
                0x00206a94                Timer0B_IRQHandler
                0x00206a94                M3FlashSingleErr_IRQHandler
                0x00206a94                I2C0_IRQHandler
                0x00206a94                ADCInt7_IRQHandler
                0x00206a94                ADCInt6_IRQHandler
                0x00206a94                PendSV_Handler
                0x00206a94                I2C1_IRQHandler
                0x00206a94                UART1_IRQHandler
                0x00206a94                ADCInt5_IRQHandler
                0x00206a94                Timer1B_IRQHandler
                0x00206a94                Watchdog_IRQHandler
                0x00206a94                EPI_IRQHandler
                0x00206a94                UART0_IRQHandler
                0x00206a94                SSI0_IRQHandler
                0x00206a94                sys_usb_pll_ofl_IRQHandler
                0x00206a94                SSI1_IRQHandler
                0x00206a94                ADCInt8_IRQHandler
                0x00206a94                GPIOPortC_IRQHandler
                0x00206a94                UART2_IRQHandler
                0x00206a94                UART4_IRQHandler
                0x00206a94                uDMAerr_IRQHandler
                0x00206a94                GPIOPortJ_IRQHandler
                0x00206a94                CAN1Init1_IRQHandler
                0x00206a94                Default_Handler
                0x00206a94                CAN0Init0_IRQHandler
                0x00206a94                USB_IRQHandler
                0x00206a94                GPIOPortD_IRQHandler
                0x00206a94                SVC_Handler
                0x00206a94                Timer3B_IRQHandler
                0x00206a94                Timer3A_IRQHandler
                0x00206a94                GPIOPortA_IRQHandler
                0x00206a94                CAN1Init0_IRQHandler
                0x00206a94                Timer0A_IRQHandler
                0x00206a94                ADCInt1_IRQHandler
                0x00206a94                Timer1A_IRQHandler
                0x00206a94                GPIOPortG_IRQHandler
                0x00206a94                CTOMIPC3_IRQHandler
                0x00206a94                ADCInt3_IRQHandler
                0x00206a94                uDMAsoft_IRQHandler
                0x00206a94                ETH_IRQHandler
                0x00206a94                GPIOPortE_IRQHandler
                0x00206a94                CTOMIPC1_IRQHandler
                0x00206a94                CAN0Init1_IRQHandler
                0x00206a94                SSI2_IRQHandler
                0x00206a94                GPIOPortF_IRQHandler
                0x00206a94                ADCInt2_IRQHandler
                0x00206a94                GPIOPortB_IRQHandler
                0x00206a94                GPIOPortH_IRQHandler
                0x00206a94                Timer2A_IRQHandler
                0x00206a94                SSI3_IRQHandler
                0x00206a94                Timer2B_IRQHandler
                0x00206a94                ADCInt4_IRQHandler
                0x00206a94                UART3_IRQHandler
                0x00206a94                SysCtrl_IRQHandler
                0x00206a94                RamSingleErr_IRQHandler
                0x00206a94                CTOMIPC4_IRQHandler
 .text          0x00206ac0     0x101c ./sysctl.o
                0x00206ac0                SysCtlSRAMSizeGet
                0x00206b08                SysCtlFlashSizeGet
                0x00206b24                SysCtlPeripheralPresent
                0x00206bec                SysCtlPeripheralReset
                0x00206d14                SysCtlPeripheralEnable
                0x00206d6c                SysCtlPeripheralDisable
                0x00206dc8                SysCtlPeripheralIsEnabled
                0x00206e08                SysCtlPeripheralSleepEnable
                0x00206e60                SysCtlPeripheralSleepDisable
                0x00206ebc                SysCtlPeripheralDeepSleepEnable
                0x00206f14                SysCtlPeripheralDeepSleepDisable
                0x00206f70                SysCtlPeripheralClockGating
                0x00206fc0                SysCtlReset
                0x00206fd4                SysCtlSleep
                0x00206fe0                SysCtlDeepSleep
                0x00207008                SysCtlResetCauseGet
                0x00207020                SysCtlResetCauseClear
                0x00207044                SysCtlDelay
                0x00207074                SysCtlXPllClockDividerSet
                0x00207110                SysCtlClockDividersSet
                0x00207268                SysCtlPowerOffPLL
                0x002072a0                SysCtlClockPllConfig
                0x0020745c                SysCtlClockConfigSet
                0x002074b8                SysCtlClockConfigGet
                0x00207554                SysCtlClockGet
                0x00207630                SysCtlC28Enable
                0x00207668                SysCtlC28Disable
                0x002076a0                SysCtlGPIOAHBEnable
                0x002076e0                SysCtlGPIOAHBDisable
                0x00207720                SysCtlUSBPLLEnable
                0x0020777c                SysCtlUSBPLLDisable
                0x002077b4                SysCtlUSBPLLConfigSet
                0x00207898                SysCtlUSBPLLConfigGet
                0x002078dc                SysCtlEnableAERRNMI
                0x00207910                SysCtlGetNmiConfig
                0x00207928                SysCtlGetNmiInterruptStatus
                0x0020794c                SysCtlGetNmiFlagStatus
                0x00207964                SysCtlNmiIsSet
                0x00207990                SysCtlNmiFlgClr
                0x002079c8                SysCtlNmiFlgClrAll
                0x00207a00                SysCtlHoldSubSystemInReset
                0x00207a44                SysCtlReleaseSubSystemFromReset
                0x00207a84                SysCtlSubSystemReset
 .text          0x00207adc        0x0 ./system_F28M35H2C.o
 .text          0x00207adc      0x104 ./systick.o
                0x00207adc                SysTickEnable
                0x00207af8                SysTickDisable
                0x00207b14                SysTickIntRegister
                0x00207b3c                SysTickIntUnregister
                0x00207b58                SysTickIntEnable
                0x00207b74                SysTickIntDisable
                0x00207b90                SysTickPeriodSet
                0x00207bb0                SysTickPeriodGet
                0x00207bc8                SysTickValueGet
 .text          0x00207be0      0x23c ./watchdog.o
                0x00207be0                WatchdogRunning
                0x00207c04                WatchdogEnable
                0x00207c28                WatchdogResetEnable
                0x00207c4c                WatchdogResetDisable
                0x00207c70                WatchdogLock
                0x00207c8c                WatchdogUnlock
                0x00207cac                WatchdogLockState
                0x00207cd4                WatchdogReloadSet
                0x00207cf0                WatchdogReloadGet
                0x00207d08                WatchdogValueGet
                0x00207d24                WatchdogIntRegister
                0x00207d44                WatchdogIntUnregister
                0x00207d60                WatchdogIntEnable
                0x00207d84                WatchdogIntStatus
                0x00207db0                WatchdogIntClear
                0x00207dcc                WatchdogStallEnable
                0x00207df4                WatchdogStallDisable
 .text          0x00207e1c        0x0 /opt/ic-dev-env/gcc-arm-none-eabi-4_8-2014q3/bin/../lib/gcc/arm-none-eabi/4.8.4/../../../../arm-none-eabi/lib/armv7-m/libc.a(lib_a-exit.o)
 .text          0x00207e1c        0x0 /opt/ic-dev-env/gcc-arm-none-eabi-4_8-2014q3/bin/../lib/gcc/arm-none-eabi/4.8.4/../../../../arm-none-eabi/lib/armv7-m/libc.a(lib_a-impure.o)
 .text          0x00207e1c        0x0 /opt/ic-dev-env/gcc-arm-none-eabi-4_8-2014q3/bin/../lib/gcc/arm-none-eabi/4.8.4/../../../../arm-none-eabi/lib/armv7-m/libc.a(lib_a-init.o)
 .text          0x00207e1c       0xec /opt/ic-dev-env/gcc-arm-none-eabi-4_8-2014q3/bin/../lib/gcc/arm-none-eabi/4.8.4/../../../../arm-none-eabi/lib/armv7-m/libc.a(lib_a-memcpy.o)
                0x00207e1c                memcpy
 .text          0x00207f08        0x0 /opt/ic-dev-env/gcc-arm-none-eabi-4_8-2014q3/bin/../lib/gcc/arm-none-eabi/4.8.4/../../../../arm-none-eabi/lib/armv7-m/libc.a(lib_a-memset.o)
 .text          0x00207f08        0x0 /opt/ic-dev-env/gcc-arm-none-eabi-4_8-2014q3/bin/../lib/gcc/arm-none-eabi/4.8.4/../../../../arm-none-eabi/lib/armv7-m/libc.a(lib_a-__call_atexit.o)
 .text          0x00207f08        0x0 /opt/ic-dev-env/gcc-arm-none-eabi-4_8-2014q3/bin/../lib/gcc/arm-none-eabi/4.8.4/../../../../arm-none-eabi/lib/armv7-m/libc.a(lib_a-atexit.o)
 .text          0x00207f08        0x0 /opt/ic-dev-env/gcc-arm-none-eabi-4_8-2014q3/bin/../lib/gcc/arm-none-eabi/4.8.4/../../../../arm-none-eabi/lib/armv7-m/libc.a(lib_a-fini.o)
 .text          0x00207f08        0x0 /opt/ic-dev-env/gcc-arm-none-eabi-4_8-2014q3/bin/../lib/gcc/arm-none-eabi/4.8.4/../../../../arm-none-eabi/lib/armv7-m/libc.a(lib_a-__atexit.o)
 .text          0x00207f08        0x0 /opt/ic-dev-env/gcc-arm-none-eabi-4_8-2014q3/bin/../lib/gcc/arm-none-eabi/4.8.4/../../../../arm-none-eabi/lib/armv7-m/librdimon.a(rdimon-_exit.o)
 .text          0x00207f08        0x0 /opt/ic-dev-env/gcc-arm-none-eabi-4_8-2014q3/bin/../lib/gcc/arm-none-eabi/4.8.4/../../../../arm-none-eabi/lib/armv7-m/librdimon.a(rdimon-_kill.o)
 .text          0x00207f08        0x0 /opt/ic-dev-env/gcc-arm-none-eabi-4_8-2014q3/bin/../lib/gcc/arm-none-eabi/4.8.4/armv7-m/crtend.o
 .text          0x00207f08        0x0 /opt/ic-dev-env/gcc-arm-none-eabi-4_8-2014q3/bin/../lib/gcc/arm-none-eabi/4.8.4/armv7-m/crtn.o
 *(.text*)
 .text.exit     0x00207f08       0x20 /opt/ic-dev-env/gcc-arm-none-eabi-4_8-2014q3/bin/../lib/gcc/arm-none-eabi/4.8.4/../../../../arm-none-eabi/lib/armv7-m/libc.a(lib_a-exit.o)
                0x00207f08                exit
 .text.__libc_init_array
                0x00207f28       0x50 /opt/ic-dev-env/gcc-arm-none-eabi-4_8-2014q3/bin/../lib/gcc/arm-none-eabi/4.8.4/../../../../arm-none-eabi/lib/armv7-m/libc.a(lib_a-init.o)
                0x00207f28                __libc_init_array
 .text.memset   0x00207f78       0x94 /opt/ic-dev-env/gcc-arm-none-eabi-4_8-2014q3/bin/../lib/gcc/arm-none-eabi/4.8.4/../../../../arm-none-eabi/lib/armv7-m/libc.a(lib_a-memset.o)
                0x00207f78                memset
 .text.startup.register_fini
                0x0020800c       0x14 /opt/ic-dev-env/gcc-arm-none-eabi-4_8-2014q3/bin/../lib/gcc/arm-none-eabi/4.8.4/../../../../arm-none-eabi/lib/armv7-m/libc.a(lib_a-__call_atexit.o)
 .text.__call_exitprocs
                0x00208020       0xf0 /opt/ic-dev-env/gcc-arm-none-eabi-4_8-2014q3/bin/../lib/gcc/arm-none-eabi/4.8.4/../../../../arm-none-eabi/lib/armv7-m/libc.a(lib_a-__call_atexit.o)
                0x00208020                __call_exitprocs
 .text.atexit   0x00208110        0xc /opt/ic-dev-env/gcc-arm-none-eabi-4_8-2014q3/bin/../lib/gcc/arm-none-eabi/4.8.4/../../../../arm-none-eabi/lib/armv7-m/libc.a(lib_a-atexit.o)
                0x00208110                atexit
 .text.__libc_fini_array
                0x0020811c       0x30 /opt/ic-dev-env/gcc-arm-none-eabi-4_8-2014q3/bin/../lib/gcc/arm-none-eabi/4.8.4/../../../../arm-none-eabi/lib/armv7-m/libc.a(lib_a-fini.o)
                0x0020811c                __libc_fini_array
 .text.__register_exitproc
                0x0020814c       0xa8 /opt/ic-dev-env/gcc-arm-none-eabi-4_8-2014q3/bin/../lib/gcc/arm-none-eabi/4.8.4/../../../../arm-none-eabi/lib/armv7-m/libc.a(lib_a-__atexit.o)
                0x0020814c                __register_exitproc
 .text._exit    0x002081f4        0x8 /opt/ic-dev-env/gcc-arm-none-eabi-4_8-2014q3/bin/../lib/gcc/arm-none-eabi/4.8.4/../../../../arm-none-eabi/lib/armv7-m/librdimon.a(rdimon-_exit.o)
                0x002081f4                _exit
 .text._kill    0x002081fc       0x20 /opt/ic-dev-env/gcc-arm-none-eabi-4_8-2014q3/bin/../lib/gcc/arm-none-eabi/4.8.4/../../../../arm-none-eabi/lib/armv7-m/librdimon.a(rdimon-_kill.o)
                0x002081fc                _kill
 *(.rodata)
 .rodata        0x0020821c       0x88 ./gpio.o
 .rodata        0x002082a4       0x68 ./interrupt.o
 .rodata        0x0020830c       0x10 ./startup_ccs.o
 .rodata        0x0020831c       0x64 ./sysctl.o
 *(.rodata*)
 .rodata.str1.4
                0x00208380        0x4 /opt/ic-dev-env/gcc-arm-none-eabi-4_8-2014q3/bin/../lib/gcc/arm-none-eabi/4.8.4/../../../../arm-none-eabi/lib/armv7-m/libc.a(lib_a-impure.o)
 .rodata._global_impure_ptr
                0x00208384        0x4 /opt/ic-dev-env/gcc-arm-none-eabi-4_8-2014q3/bin/../lib/gcc/arm-none-eabi/4.8.4/../../../../arm-none-eabi/lib/armv7-m/libc.a(lib_a-impure.o)
                0x00208384                _global_impure_ptr
 *(.init)
 .init          0x00208388        0x4 /opt/ic-dev-env/gcc-arm-none-eabi-4_8-2014q3/bin/../lib/gcc/arm-none-eabi/4.8.4/armv7-m/crti.o
                0x00208388                _init
 .init          0x0020838c        0x8 /opt/ic-dev-env/gcc-arm-none-eabi-4_8-2014q3/bin/../lib/gcc/arm-none-eabi/4.8.4/armv7-m/crtn.o
 *(.fini)
 .fini          0x00208394        0x4 /opt/ic-dev-env/gcc-arm-none-eabi-4_8-2014q3/bin/../lib/gcc/arm-none-eabi/4.8.4/armv7-m/crti.o
                0x00208394                _fini
 .fini          0x00208398        0x8 /opt/ic-dev-env/gcc-arm-none-eabi-4_8-2014q3/bin/../lib/gcc/arm-none-eabi/4.8.4/armv7-m/crtn.o
                0x002083a0                . = ALIGN (0x4)

.glue_7         0x002083a0        0x0
 .glue_7        0x00000000        0x0 linker stubs

.glue_7t        0x002083a0        0x0
 .glue_7t       0x00000000        0x0 linker stubs

.vfp11_veneer   0x002083a0        0x0
 .vfp11_veneer  0x00000000        0x0 linker stubs

.v4_bx          0x002083a0        0x0
 .v4_bx         0x00000000        0x0 linker stubs

.iplt           0x002083a0        0x0
 .iplt          0x00000000        0x0 /opt/ic-dev-env/gcc-arm-none-eabi-4_8-2014q3/bin/../lib/gcc/arm-none-eabi/4.8.4/armv7-m/crtbegin.o

.preinit_array  0x002083a0        0x0
                0x002083a0                PROVIDE (__preinit_array_start, .)
 *(.preinit_array*)
                0x002083a0                PROVIDE (__preinit_array_end, .)

.init_array     0x002083a0        0x8
                0x002083a0                PROVIDE (__init_array_start, .)
 *(SORT(.init_array.*))
 .init_array.00000
                0x002083a0        0x4 /opt/ic-dev-env/gcc-arm-none-eabi-4_8-2014q3/bin/../lib/gcc/arm-none-eabi/4.8.4/../../../../arm-none-eabi/lib/armv7-m/libc.a(lib_a-__call_atexit.o)
 *(.init_array*)
 .init_array    0x002083a4        0x4 /opt/ic-dev-env/gcc-arm-none-eabi-4_8-2014q3/bin/../lib/gcc/arm-none-eabi/4.8.4/armv7-m/crtbegin.o
                0x002083a8                PROVIDE (__init_array_end, .)

.fini_array     0x002083a8        0x4
                0x002083a8                PROVIDE (__fini_array_start, .)
 *(.fini_array*)
 .fini_array    0x002083a8        0x4 /opt/ic-dev-env/gcc-arm-none-eabi-4_8-2014q3/bin/../lib/gcc/arm-none-eabi/4.8.4/armv7-m/crtbegin.o
 *(SORT(.fini_array.*))
                0x002083ac                PROVIDE (__fini_array_end, .)

.flashload      0x00201200      0x134
 *(.flashload)
 .flashload     0x00201200      0x134 ./flash.o
                0x00201200                FlashInit
                0x00201298                FlashSetup
                0x00201334                . = ALIGN (0x4)
                0x00201200                RamfuncsLoadStart = LOADADDR (.flashload)
                0x00000134                RamfuncsLoadSize = SIZEOF (.flashload)
                0x00201334                _etext = .

.rel.dyn        0x00201334        0x0
 .rel.iplt      0x00000000        0x0 /opt/ic-dev-env/gcc-arm-none-eabi-4_8-2014q3/bin/../lib/gcc/arm-none-eabi/4.8.4/armv7-m/crtbegin.o

.ramfuncs       0x20000000        0x0
 *(.ramfuncs)
                0x20000000                . = ALIGN (0x4)
                0x20000000                RamfuncsRunStart = LOADADDR (.ramfuncs)

.vtable         0x20002000      0x258
 *(.vtable)
 .vtable        0x20002000      0x258 ./interrupt.o
                0x20002000                g_pfnRAMVectors
                0x20002258                . = ALIGN (0x4)

.stack          0x20002258      0x400
                0x20002258                __stack_start__ = .
                0x20002658                . = (. + STACK_SIZE)
 *fill*         0x20002258      0x400 
                0x20002658                . = ALIGN (0x4)
                0x20002658                __stack_end__ = .

.data           0x20002658      0x434 load address 0x00201334
                0x00201334                __data_load = LOADADDR (.data)
                0x20002658                __data_start = .
 *(.data)
 .data          0x20002658        0x0 /opt/ic-dev-env/gcc-arm-none-eabi-4_8-2014q3/bin/../lib/gcc/arm-none-eabi/4.8.4/armv7-m/crti.o
 .data          0x20002658        0x4 /opt/ic-dev-env/gcc-arm-none-eabi-4_8-2014q3/bin/../lib/gcc/arm-none-eabi/4.8.4/armv7-m/crtbegin.o
                0x20002658                __dso_handle
 .data          0x2000265c        0x0 /opt/ic-dev-env/gcc-arm-none-eabi-4_8-2014q3/bin/../lib/gcc/arm-none-eabi/4.8.4/../../../../arm-none-eabi/lib/armv7-m/crt0.o
 .data          0x2000265c        0x0 ./bsp.o
 .data          0x2000265c        0x0 ./cpu.o
 .data          0x2000265c        0x0 ./flash.o
 .data          0x2000265c        0x0 ./gpio.o
 .data          0x2000265c        0x0 ./interrupt.o
 .data          0x2000265c        0x0 ./ipc.o
 .data          0x2000265c        0x0 ./ipc_lite.o
 .data          0x2000265c        0x0 ./ipc_util.o
 .data          0x2000265c        0x0 ./main.o
 .data          0x2000265c        0x0 ./ram.o
 .data          0x2000265c        0x0 ./startup_ccs.o
 .data          0x2000265c        0x0 ./sysctl.o
 .data          0x2000265c        0x0 ./system_F28M35H2C.o
 .data          0x2000265c        0x0 ./systick.o
 .data          0x2000265c        0x0 ./watchdog.o
 .data          0x2000265c        0x0 /opt/ic-dev-env/gcc-arm-none-eabi-4_8-2014q3/bin/../lib/gcc/arm-none-eabi/4.8.4/../../../../arm-none-eabi/lib/armv7-m/libc.a(lib_a-exit.o)
 .data          0x2000265c        0x0 /opt/ic-dev-env/gcc-arm-none-eabi-4_8-2014q3/bin/../lib/gcc/arm-none-eabi/4.8.4/../../../../arm-none-eabi/lib/armv7-m/libc.a(lib_a-impure.o)
 .data          0x2000265c        0x0 /opt/ic-dev-env/gcc-arm-none-eabi-4_8-2014q3/bin/../lib/gcc/arm-none-eabi/4.8.4/../../../../arm-none-eabi/lib/armv7-m/libc.a(lib_a-init.o)
 .data          0x2000265c        0x0 /opt/ic-dev-env/gcc-arm-none-eabi-4_8-2014q3/bin/../lib/gcc/arm-none-eabi/4.8.4/../../../../arm-none-eabi/lib/armv7-m/libc.a(lib_a-memcpy.o)
 .data          0x2000265c        0x0 /opt/ic-dev-env/gcc-arm-none-eabi-4_8-2014q3/bin/../lib/gcc/arm-none-eabi/4.8.4/../../../../arm-none-eabi/lib/armv7-m/libc.a(lib_a-memset.o)
 .data          0x2000265c        0x0 /opt/ic-dev-env/gcc-arm-none-eabi-4_8-2014q3/bin/../lib/gcc/arm-none-eabi/4.8.4/../../../../arm-none-eabi/lib/armv7-m/libc.a(lib_a-__call_atexit.o)
 .data          0x2000265c        0x0 /opt/ic-dev-env/gcc-arm-none-eabi-4_8-2014q3/bin/../lib/gcc/arm-none-eabi/4.8.4/../../../../arm-none-eabi/lib/armv7-m/libc.a(lib_a-atexit.o)
 .data          0x2000265c        0x0 /opt/ic-dev-env/gcc-arm-none-eabi-4_8-2014q3/bin/../lib/gcc/arm-none-eabi/4.8.4/../../../../arm-none-eabi/lib/armv7-m/libc.a(lib_a-fini.o)
 .data          0x2000265c        0x0 /opt/ic-dev-env/gcc-arm-none-eabi-4_8-2014q3/bin/../lib/gcc/arm-none-eabi/4.8.4/../../../../arm-none-eabi/lib/armv7-m/libc.a(lib_a-__atexit.o)
 .data          0x2000265c        0x0 /opt/ic-dev-env/gcc-arm-none-eabi-4_8-2014q3/bin/../lib/gcc/arm-none-eabi/4.8.4/../../../../arm-none-eabi/lib/armv7-m/librdimon.a(rdimon-_exit.o)
 .data          0x2000265c        0x0 /opt/ic-dev-env/gcc-arm-none-eabi-4_8-2014q3/bin/../lib/gcc/arm-none-eabi/4.8.4/../../../../arm-none-eabi/lib/armv7-m/librdimon.a(rdimon-_kill.o)
 .data          0x2000265c        0x0 /opt/ic-dev-env/gcc-arm-none-eabi-4_8-2014q3/bin/../lib/gcc/arm-none-eabi/4.8.4/armv7-m/crtend.o
 .data          0x2000265c        0x0 /opt/ic-dev-env/gcc-arm-none-eabi-4_8-2014q3/bin/../lib/gcc/arm-none-eabi/4.8.4/armv7-m/crtn.o
 *(.data*)
 *fill*         0x2000265c        0x4 
 .data.impure_data
                0x20002660      0x428 /opt/ic-dev-env/gcc-arm-none-eabi-4_8-2014q3/bin/../lib/gcc/arm-none-eabi/4.8.4/../../../../arm-none-eabi/lib/armv7-m/libc.a(lib_a-impure.o)
 .data._impure_ptr
                0x20002a88        0x4 /opt/ic-dev-env/gcc-arm-none-eabi-4_8-2014q3/bin/../lib/gcc/arm-none-eabi/4.8.4/../../../../arm-none-eabi/lib/armv7-m/libc.a(lib_a-impure.o)
                0x20002a88                _impure_ptr
                0x20002a8c                . = ALIGN (0x4)
                0x20002a8c                __data_end__ = .
                0x20002a8c                _edata = __data_end__

.jcr            0x20002a8c        0x4 load address 0x00201768
 .jcr           0x20002a8c        0x0 /opt/ic-dev-env/gcc-arm-none-eabi-4_8-2014q3/bin/../lib/gcc/arm-none-eabi/4.8.4/armv7-m/crtbegin.o
 .jcr           0x20002a8c        0x4 /opt/ic-dev-env/gcc-arm-none-eabi-4_8-2014q3/bin/../lib/gcc/arm-none-eabi/4.8.4/armv7-m/crtend.o

.igot.plt       0x20002a90        0x0 load address 0x0020176c
 .igot.plt      0x00000000        0x0 /opt/ic-dev-env/gcc-arm-none-eabi-4_8-2014q3/bin/../lib/gcc/arm-none-eabi/4.8.4/armv7-m/crtbegin.o

.bss            0x20002a90       0x24 load address 0x0020176c
                0x20002a90                __bss_start__ = .
 *(.bss)
 .bss           0x20002a90        0x0 /opt/ic-dev-env/gcc-arm-none-eabi-4_8-2014q3/bin/../lib/gcc/arm-none-eabi/4.8.4/armv7-m/crti.o
 .bss           0x20002a90       0x1c /opt/ic-dev-env/gcc-arm-none-eabi-4_8-2014q3/bin/../lib/gcc/arm-none-eabi/4.8.4/armv7-m/crtbegin.o
 .bss           0x20002aac        0x0 /opt/ic-dev-env/gcc-arm-none-eabi-4_8-2014q3/bin/../lib/gcc/arm-none-eabi/4.8.4/../../../../arm-none-eabi/lib/armv7-m/crt0.o
 .bss           0x20002aac        0x4 ./bsp.o
                0x20002aac                TimmingDelay
 .bss           0x20002ab0        0x0 ./cpu.o
 .bss           0x20002ab0        0x0 ./flash.o
 .bss           0x20002ab0        0x0 ./gpio.o
 .bss           0x20002ab0        0x0 ./interrupt.o
 .bss           0x20002ab0        0x0 ./ipc.o
 .bss           0x20002ab0        0x0 ./ipc_lite.o
 .bss           0x20002ab0        0x0 ./ipc_util.o
 .bss           0x20002ab0        0x0 ./main.o
 .bss           0x20002ab0        0x4 ./ram.o
 .bss           0x20002ab4        0x0 ./startup_ccs.o
 .bss           0x20002ab4        0x0 ./sysctl.o
 .bss           0x20002ab4        0x0 ./system_F28M35H2C.o
 .bss           0x20002ab4        0x0 ./systick.o
 .bss           0x20002ab4        0x0 ./watchdog.o
 .bss           0x20002ab4        0x0 /opt/ic-dev-env/gcc-arm-none-eabi-4_8-2014q3/bin/../lib/gcc/arm-none-eabi/4.8.4/../../../../arm-none-eabi/lib/armv7-m/libc.a(lib_a-exit.o)
 .bss           0x20002ab4        0x0 /opt/ic-dev-env/gcc-arm-none-eabi-4_8-2014q3/bin/../lib/gcc/arm-none-eabi/4.8.4/../../../../arm-none-eabi/lib/armv7-m/libc.a(lib_a-impure.o)
 .bss           0x20002ab4        0x0 /opt/ic-dev-env/gcc-arm-none-eabi-4_8-2014q3/bin/../lib/gcc/arm-none-eabi/4.8.4/../../../../arm-none-eabi/lib/armv7-m/libc.a(lib_a-init.o)
 .bss           0x20002ab4        0x0 /opt/ic-dev-env/gcc-arm-none-eabi-4_8-2014q3/bin/../lib/gcc/arm-none-eabi/4.8.4/../../../../arm-none-eabi/lib/armv7-m/libc.a(lib_a-memcpy.o)
 .bss           0x20002ab4        0x0 /opt/ic-dev-env/gcc-arm-none-eabi-4_8-2014q3/bin/../lib/gcc/arm-none-eabi/4.8.4/../../../../arm-none-eabi/lib/armv7-m/libc.a(lib_a-memset.o)
 .bss           0x20002ab4        0x0 /opt/ic-dev-env/gcc-arm-none-eabi-4_8-2014q3/bin/../lib/gcc/arm-none-eabi/4.8.4/../../../../arm-none-eabi/lib/armv7-m/libc.a(lib_a-__call_atexit.o)
 .bss           0x20002ab4        0x0 /opt/ic-dev-env/gcc-arm-none-eabi-4_8-2014q3/bin/../lib/gcc/arm-none-eabi/4.8.4/../../../../arm-none-eabi/lib/armv7-m/libc.a(lib_a-atexit.o)
 .bss           0x20002ab4        0x0 /opt/ic-dev-env/gcc-arm-none-eabi-4_8-2014q3/bin/../lib/gcc/arm-none-eabi/4.8.4/../../../../arm-none-eabi/lib/armv7-m/libc.a(lib_a-fini.o)
 .bss           0x20002ab4        0x0 /opt/ic-dev-env/gcc-arm-none-eabi-4_8-2014q3/bin/../lib/gcc/arm-none-eabi/4.8.4/../../../../arm-none-eabi/lib/armv7-m/libc.a(lib_a-__atexit.o)
 .bss           0x20002ab4        0x0 /opt/ic-dev-env/gcc-arm-none-eabi-4_8-2014q3/bin/../lib/gcc/arm-none-eabi/4.8.4/../../../../arm-none-eabi/lib/armv7-m/librdimon.a(rdimon-_exit.o)
 .bss           0x20002ab4        0x0 /opt/ic-dev-env/gcc-arm-none-eabi-4_8-2014q3/bin/../lib/gcc/arm-none-eabi/4.8.4/../../../../arm-none-eabi/lib/armv7-m/librdimon.a(rdimon-_kill.o)
 .bss           0x20002ab4        0x0 /opt/ic-dev-env/gcc-arm-none-eabi-4_8-2014q3/bin/../lib/gcc/arm-none-eabi/4.8.4/armv7-m/crtend.o
 .bss           0x20002ab4        0x0 /opt/ic-dev-env/gcc-arm-none-eabi-4_8-2014q3/bin/../lib/gcc/arm-none-eabi/4.8.4/armv7-m/crtn.o
 *(.bss*)
 *(COMMON)
                0x20002ab4                . = ALIGN (0x4)
                0x20002ab4                _ebss = .
                0x20002ab4                __bss_end__ = .
                0x20002ab4                PROVIDE (end, _ebss)
                0x20002ab4                PROVIDE (_end, _ebss)
                0x20002ab4                PROVIDE (__end__, _ebss)

.heap           0x20002ab4      0x100 load address 0x00201790
                0x20002ab4                __heap_start__ = .
                0x20002bb4                . = (. + HEAP_SIZE)
 *fill*         0x20002ab4      0x100 
                0x20002bb4                . = ALIGN (0x4)
                0x20002bb4                __heap_end__ = .

PUTBUFFER       0x2007f800      0x100
 *(PUTBUFFER)
 PUTBUFFER      0x2007f800      0x100 ./ipc.o
                0x2007f800                g_asIPCMtoCBuffers
                0x2007f900                . = ALIGN (0x4)

PUTWRITEIDX     0x2007f900        0x8
 *(PUTWRITEIDX)
 PUTWRITEIDX    0x2007f900        0x8 ./ipc.o
                0x2007f900                g_usPutWriteIndexes
                0x2007f908                . = ALIGN (0x4)

GETREADIDX      0x2007f908        0x8
 *(GETREADIDX)
 GETREADIDX     0x2007f908        0x8 ./ipc.o
                0x2007f908                g_usGetReadIndexes
                0x2007f910                . = ALIGN (0x4)

GETBUFFER       0x2007f000      0x100
 *(GETBUFFER)
 GETBUFFER      0x2007f000      0x100 ./ipc.o
                0x2007f000                g_asIPCCtoMBuffers
                0x2007f100                . = ALIGN (0x4)

GETWRITEIDX     0x2007f100        0x8
 *(GETWRITEIDX)
 GETWRITEIDX    0x2007f100        0x8 ./ipc.o
                0x2007f100                g_usGetWriteIndexes
                0x2007f108                . = ALIGN (0x4)

PUTREADIDX      0x2007f108        0x8
 *(PUTREADIDX)
 PUTREADIDX     0x2007f108        0x8 ./ipc.o
                0x2007f108                g_usPutReadIndexes
                0x2007f110                . = ALIGN (0x4)
LOAD /home/preetham/controlSUITE/device_support/f28m35x/v207/MWare/driverlib/ccs/Debug/driverlib.lib
START GROUP
LOAD /opt/ic-dev-env/gcc-arm-none-eabi-4_8-2014q3/bin/../lib/gcc/arm-none-eabi/4.8.4/../../../../arm-none-eabi/lib/armv7-m/libc.a
LOAD /opt/ic-dev-env/gcc-arm-none-eabi-4_8-2014q3/bin/../lib/gcc/arm-none-eabi/4.8.4/../../../../arm-none-eabi/lib/armv7-m/libm.a
LOAD /opt/ic-dev-env/gcc-arm-none-eabi-4_8-2014q3/bin/../lib/gcc/arm-none-eabi/4.8.4/armv7-m/libgcc.a
LOAD /opt/ic-dev-env/gcc-arm-none-eabi-4_8-2014q3/bin/../lib/gcc/arm-none-eabi/4.8.4/../../../../arm-none-eabi/lib/armv7-m/libnosys.a
END GROUP
START GROUP
LOAD /opt/ic-dev-env/gcc-arm-none-eabi-4_8-2014q3/bin/../lib/gcc/arm-none-eabi/4.8.4/armv7-m/libgcc.a
LOAD /opt/ic-dev-env/gcc-arm-none-eabi-4_8-2014q3/bin/../lib/gcc/arm-none-eabi/4.8.4/../../../../arm-none-eabi/lib/armv7-m/libg.a
LOAD /opt/ic-dev-env/gcc-arm-none-eabi-4_8-2014q3/bin/../lib/gcc/arm-none-eabi/4.8.4/../../../../arm-none-eabi/lib/armv7-m/libc.a
END GROUP
LOAD /opt/ic-dev-env/gcc-arm-none-eabi-4_8-2014q3/bin/../lib/gcc/arm-none-eabi/4.8.4/armv7-m/crtend.o
LOAD /opt/ic-dev-env/gcc-arm-none-eabi-4_8-2014q3/bin/../lib/gcc/arm-none-eabi/4.8.4/armv7-m/crtn.o
OUTPUT(Test.out elf32-littlearm)

.ARM.attributes
                0x00000000       0x29
 .ARM.attributes
                0x00000000       0x1d /opt/ic-dev-env/gcc-arm-none-eabi-4_8-2014q3/bin/../lib/gcc/arm-none-eabi/4.8.4/armv7-m/crti.o
 .ARM.attributes
                0x0000001d       0x2d /opt/ic-dev-env/gcc-arm-none-eabi-4_8-2014q3/bin/../lib/gcc/arm-none-eabi/4.8.4/armv7-m/crtbegin.o
 .ARM.attributes
                0x0000004a       0x1b /opt/ic-dev-env/gcc-arm-none-eabi-4_8-2014q3/bin/../lib/gcc/arm-none-eabi/4.8.4/../../../../arm-none-eabi/lib/armv7-m/crt0.o
 .ARM.attributes
                0x00000065       0x33 ./bsp.o
 .ARM.attributes
                0x00000098       0x33 ./cpu.o
 .ARM.attributes
                0x000000cb       0x33 ./flash.o
 .ARM.attributes
                0x000000fe       0x33 ./gpio.o
 .ARM.attributes
                0x00000131       0x33 ./interrupt.o
 .ARM.attributes
                0x00000164       0x33 ./ipc.o
 .ARM.attributes
                0x00000197       0x33 ./ipc_lite.o
 .ARM.attributes
                0x000001ca       0x33 ./ipc_util.o
 .ARM.attributes
                0x000001fd       0x33 ./main.o
 .ARM.attributes
                0x00000230       0x33 ./ram.o
 .ARM.attributes
                0x00000263       0x33 ./startup_ccs.o
 .ARM.attributes
                0x00000296       0x33 ./sysctl.o
 .ARM.attributes
                0x000002c9       0x33 ./system_F28M35H2C.o
 .ARM.attributes
                0x000002fc       0x33 ./systick.o
 .ARM.attributes
                0x0000032f       0x33 ./watchdog.o
 .ARM.attributes
                0x00000362       0x2d /opt/ic-dev-env/gcc-arm-none-eabi-4_8-2014q3/bin/../lib/gcc/arm-none-eabi/4.8.4/../../../../arm-none-eabi/lib/armv7-m/libc.a(lib_a-exit.o)
 .ARM.attributes
                0x0000038f       0x2d /opt/ic-dev-env/gcc-arm-none-eabi-4_8-2014q3/bin/../lib/gcc/arm-none-eabi/4.8.4/../../../../arm-none-eabi/lib/armv7-m/libc.a(lib_a-impure.o)
 .ARM.attributes
                0x000003bc       0x2d /opt/ic-dev-env/gcc-arm-none-eabi-4_8-2014q3/bin/../lib/gcc/arm-none-eabi/4.8.4/../../../../arm-none-eabi/lib/armv7-m/libc.a(lib_a-init.o)
 .ARM.attributes
                0x000003e9       0x1b /opt/ic-dev-env/gcc-arm-none-eabi-4_8-2014q3/bin/../lib/gcc/arm-none-eabi/4.8.4/../../../../arm-none-eabi/lib/armv7-m/libc.a(lib_a-memcpy.o)
 .ARM.attributes
                0x00000404       0x2d /opt/ic-dev-env/gcc-arm-none-eabi-4_8-2014q3/bin/../lib/gcc/arm-none-eabi/4.8.4/../../../../arm-none-eabi/lib/armv7-m/libc.a(lib_a-memset.o)
 .ARM.attributes
                0x00000431       0x2d /opt/ic-dev-env/gcc-arm-none-eabi-4_8-2014q3/bin/../lib/gcc/arm-none-eabi/4.8.4/../../../../arm-none-eabi/lib/armv7-m/libc.a(lib_a-__call_atexit.o)
 .ARM.attributes
                0x0000045e       0x2d /opt/ic-dev-env/gcc-arm-none-eabi-4_8-2014q3/bin/../lib/gcc/arm-none-eabi/4.8.4/../../../../arm-none-eabi/lib/armv7-m/libc.a(lib_a-atexit.o)
 .ARM.attributes
                0x0000048b       0x2d /opt/ic-dev-env/gcc-arm-none-eabi-4_8-2014q3/bin/../lib/gcc/arm-none-eabi/4.8.4/../../../../arm-none-eabi/lib/armv7-m/libc.a(lib_a-fini.o)
 .ARM.attributes
                0x000004b8       0x2d /opt/ic-dev-env/gcc-arm-none-eabi-4_8-2014q3/bin/../lib/gcc/arm-none-eabi/4.8.4/../../../../arm-none-eabi/lib/armv7-m/libc.a(lib_a-__atexit.o)
 .ARM.attributes
                0x000004e5       0x2d /opt/ic-dev-env/gcc-arm-none-eabi-4_8-2014q3/bin/../lib/gcc/arm-none-eabi/4.8.4/../../../../arm-none-eabi/lib/armv7-m/librdimon.a(rdimon-_exit.o)
 .ARM.attributes
                0x00000512       0x2d /opt/ic-dev-env/gcc-arm-none-eabi-4_8-2014q3/bin/../lib/gcc/arm-none-eabi/4.8.4/../../../../arm-none-eabi/lib/armv7-m/librdimon.a(rdimon-_kill.o)
 .ARM.attributes
                0x0000053f       0x2d /opt/ic-dev-env/gcc-arm-none-eabi-4_8-2014q3/bin/../lib/gcc/arm-none-eabi/4.8.4/armv7-m/crtend.o
 .ARM.attributes
                0x0000056c       0x1d /opt/ic-dev-env/gcc-arm-none-eabi-4_8-2014q3/bin/../lib/gcc/arm-none-eabi/4.8.4/armv7-m/crtn.o

.comment        0x00000000       0x70
 .comment       0x00000000       0x70 ./bsp.o
                                 0x71 (size before relaxing)
 .comment       0x00000000       0x71 ./cpu.o
 .comment       0x00000000       0x71 ./flash.o
 .comment       0x00000000       0x71 ./gpio.o
 .comment       0x00000000       0x71 ./interrupt.o
 .comment       0x00000000       0x71 ./ipc.o
 .comment       0x00000000       0x71 ./ipc_lite.o
 .comment       0x00000000       0x71 ./ipc_util.o
 .comment       0x00000000       0x71 ./main.o
 .comment       0x00000000       0x71 ./ram.o
 .comment       0x00000000       0x71 ./startup_ccs.o
 .comment       0x00000000       0x71 ./sysctl.o
 .comment       0x00000000       0x71 ./system_F28M35H2C.o
 .comment       0x00000000       0x71 ./systick.o
 .comment       0x00000000       0x71 ./watchdog.o

.debug_info     0x00000000     0x3a7b
 .debug_info    0x00000000      0x3b4 ./bsp.o
 .debug_info    0x000003b4       0xc2 ./cpu.o
 .debug_info    0x00000476       0xd9 ./flash.o
 .debug_info    0x0000054f      0x816 ./gpio.o
 .debug_info    0x00000d65      0x360 ./interrupt.o
 .debug_info    0x000010c5      0xe6d ./ipc.o
 .debug_info    0x00001f32      0x6ba ./ipc_lite.o
 .debug_info    0x000025ec      0x151 ./ipc_util.o
 .debug_info    0x0000273d       0xfe ./main.o
 .debug_info    0x0000283b       0xd5 ./ram.o
 .debug_info    0x00002910      0x41d ./startup_ccs.o
 .debug_info    0x00002d2d      0x922 ./sysctl.o
 .debug_info    0x0000364f      0x115 ./systick.o
 .debug_info    0x00003764      0x317 ./watchdog.o

.debug_abbrev   0x00000000      0xc49
 .debug_abbrev  0x00000000      0x137 ./bsp.o
 .debug_abbrev  0x00000137       0x71 ./cpu.o
 .debug_abbrev  0x000001a8       0x8d ./flash.o
 .debug_abbrev  0x00000235      0x108 ./gpio.o
 .debug_abbrev  0x0000033d      0x155 ./interrupt.o
 .debug_abbrev  0x00000492      0x144 ./ipc.o
 .debug_abbrev  0x000005d6       0xe2 ./ipc_lite.o
 .debug_abbrev  0x000006b8       0x75 ./ipc_util.o
 .debug_abbrev  0x0000072d       0x97 ./main.o
 .debug_abbrev  0x000007c4       0x93 ./ram.o
 .debug_abbrev  0x00000857      0x146 ./startup_ccs.o
 .debug_abbrev  0x0000099d      0x15c ./sysctl.o
 .debug_abbrev  0x00000af9       0x81 ./systick.o
 .debug_abbrev  0x00000b7a       0xcf ./watchdog.o

.debug_aranges  0x00000000      0x1d8
 .debug_aranges
                0x00000000       0x20 ./bsp.o
 .debug_aranges
                0x00000020       0x20 ./cpu.o
 .debug_aranges
                0x00000040       0x30 ./flash.o
 .debug_aranges
                0x00000070       0x20 ./gpio.o
 .debug_aranges
                0x00000090       0x20 ./interrupt.o
 .debug_aranges
                0x000000b0       0x20 ./ipc.o
 .debug_aranges
                0x000000d0       0x20 ./ipc_lite.o
 .debug_aranges
                0x000000f0       0x20 ./ipc_util.o
 .debug_aranges
                0x00000110       0x20 ./main.o
 .debug_aranges
                0x00000130       0x20 ./ram.o
 .debug_aranges
                0x00000150       0x28 ./startup_ccs.o
 .debug_aranges
                0x00000178       0x20 ./sysctl.o
 .debug_aranges
                0x00000198       0x20 ./systick.o
 .debug_aranges
                0x000001b8       0x20 ./watchdog.o

.debug_line     0x00000000      0xf97
 .debug_line    0x00000000      0x16e ./bsp.o
 .debug_line    0x0000016e       0x4d ./cpu.o
 .debug_line    0x000001bb       0x86 ./flash.o
 .debug_line    0x00000241      0x195 ./gpio.o
 .debug_line    0x000003d6      0x105 ./interrupt.o
 .debug_line    0x000004db      0x1d1 ./ipc.o
 .debug_line    0x000006ac      0x182 ./ipc_lite.o
 .debug_line    0x0000082e       0x89 ./ipc_util.o
 .debug_line    0x000008b7      0x13e ./main.o
 .debug_line    0x000009f5       0x76 ./ram.o
 .debug_line    0x00000a6b      0x15e ./startup_ccs.o
 .debug_line    0x00000bc9      0x2be ./sysctl.o
 .debug_line    0x00000e87        0x0 ./system_F28M35H2C.o
 .debug_line    0x00000e87       0x68 ./systick.o
 .debug_line    0x00000eef       0xa8 ./watchdog.o

.debug_str      0x00000000     0x174f
 .debug_str     0x00000000      0x250 ./bsp.o
                                0x2a8 (size before relaxing)
 .debug_str     0x00000250       0x56 ./cpu.o
                                0x123 (size before relaxing)
 .debug_str     0x000002a6       0x59 ./flash.o
                                0x154 (size before relaxing)
 .debug_str     0x000002ff      0x2fa ./gpio.o
                                0x3f1 (size before relaxing)
 .debug_str     0x000005f9      0x171 ./interrupt.o
                                0x296 (size before relaxing)
 .debug_str     0x0000076a      0x48f ./ipc.o
                                0x599 (size before relaxing)
 .debug_str     0x00000bf9      0x1eb ./ipc_lite.o
                                0x347 (size before relaxing)
 .debug_str     0x00000de4       0xa9 ./ipc_util.o
                                0x1a6 (size before relaxing)
 .debug_str     0x00000e8d       0x50 ./main.o
                                0x1bc (size before relaxing)
 .debug_str     0x00000edd       0x56 ./ram.o
                                0x163 (size before relaxing)
 .debug_str     0x00000f33      0x110 ./startup_ccs.o
                                0x30d (size before relaxing)
 .debug_str     0x00001043      0x511 ./sysctl.o
                                0x610 (size before relaxing)
 .debug_str     0x00001554        0x0 ./system_F28M35H2C.o
 .debug_str     0x00001554       0xb0 ./systick.o
                                0x196 (size before relaxing)
 .debug_str     0x00001604      0x14b ./watchdog.o
                                0x249 (size before relaxing)

.debug_frame    0x00000000     0x1874
 .debug_frame   0x00000000       0xf8 ./bsp.o
 .debug_frame   0x000000f8       0xa4 ./cpu.o
 .debug_frame   0x0000019c       0x78 ./flash.o
 .debug_frame   0x00000214      0x3b0 ./gpio.o
 .debug_frame   0x000005c4      0x1e4 ./interrupt.o
 .debug_frame   0x000007a8      0x368 ./ipc.o
 .debug_frame   0x00000b10      0x20c ./ipc_lite.o
 .debug_frame   0x00000d1c       0xd8 ./ipc_util.o
 .debug_frame   0x00000df4       0x2c ./main.o
 .debug_frame   0x00000e20       0x6c ./ram.o
 .debug_frame   0x00000e8c       0xa8 ./startup_ccs.o
 .debug_frame   0x00000f34      0x4c4 ./sysctl.o
 .debug_frame   0x000013f8       0xf8 ./systick.o
 .debug_frame   0x000014f0      0x1f4 ./watchdog.o
 .debug_frame   0x000016e4       0x28 /opt/ic-dev-env/gcc-arm-none-eabi-4_8-2014q3/bin/../lib/gcc/arm-none-eabi/4.8.4/../../../../arm-none-eabi/lib/armv7-m/libc.a(lib_a-exit.o)
 .debug_frame   0x0000170c       0x2c /opt/ic-dev-env/gcc-arm-none-eabi-4_8-2014q3/bin/../lib/gcc/arm-none-eabi/4.8.4/../../../../arm-none-eabi/lib/armv7-m/libc.a(lib_a-init.o)
 .debug_frame   0x00001738       0x2c /opt/ic-dev-env/gcc-arm-none-eabi-4_8-2014q3/bin/../lib/gcc/arm-none-eabi/4.8.4/../../../../arm-none-eabi/lib/armv7-m/libc.a(lib_a-memset.o)
 .debug_frame   0x00001764       0x48 /opt/ic-dev-env/gcc-arm-none-eabi-4_8-2014q3/bin/../lib/gcc/arm-none-eabi/4.8.4/../../../../arm-none-eabi/lib/armv7-m/libc.a(lib_a-__call_atexit.o)
 .debug_frame   0x000017ac       0x20 /opt/ic-dev-env/gcc-arm-none-eabi-4_8-2014q3/bin/../lib/gcc/arm-none-eabi/4.8.4/../../../../arm-none-eabi/lib/armv7-m/libc.a(lib_a-atexit.o)
 .debug_frame   0x000017cc       0x2c /opt/ic-dev-env/gcc-arm-none-eabi-4_8-2014q3/bin/../lib/gcc/arm-none-eabi/4.8.4/../../../../arm-none-eabi/lib/armv7-m/libc.a(lib_a-fini.o)
 .debug_frame   0x000017f8       0x30 /opt/ic-dev-env/gcc-arm-none-eabi-4_8-2014q3/bin/../lib/gcc/arm-none-eabi/4.8.4/../../../../arm-none-eabi/lib/armv7-m/libc.a(lib_a-__atexit.o)
 .debug_frame   0x00001828       0x20 /opt/ic-dev-env/gcc-arm-none-eabi-4_8-2014q3/bin/../lib/gcc/arm-none-eabi/4.8.4/../../../../arm-none-eabi/lib/armv7-m/librdimon.a(rdimon-_exit.o)
 .debug_frame   0x00001848       0x2c /opt/ic-dev-env/gcc-arm-none-eabi-4_8-2014q3/bin/../lib/gcc/arm-none-eabi/4.8.4/../../../../arm-none-eabi/lib/armv7-m/librdimon.a(rdimon-_kill.o)

.debug_ranges   0x00000000       0x38
 .debug_ranges  0x00000000       0x20 ./flash.o
 .debug_ranges  0x00000020       0x18 ./startup_ccs.o
